:020000040800F2
:10000000080F00204D010008A11A0008A31A0008DB
:10001000C91A0008CD1A0008D11A00080000000013
:100020000000000000000000000000005F01000868
:10003000D51A0008000000006301000865010008EF
:1000400067010008670100086701000867010008F0
:1000500067010008670100086701000867010008E0
:1000600067010008670100086701000867010008D0
:1000700067010008670100086701000867010008C0
:1000800067010008670100086701000867010008B0
:1000900067010008670100086701000867010008A0
:1000A0006701000867010008670100086701000890
:1000B0006701000867010008670100086701000880
:1000C0006701000867010008670100086701000870
:1000D00067010008D92600086701000867010008C9
:1000E0006701000867010008670100086701000850
:1000F0006701000867010008670100086701000840
:10010000670100082D230008670100086701000847
:10011000670100086701000867010008670100081F
:1001200067010008DFF80CD005F030FC00480047FC
:10013000CD160008080F002040BA7047C0BA7047BB
:1001400030BF72B662B680F30888704706488047B1
:1001500006480047FEE7FEE7FEE7FEE7FEE7FEE7AC
:10016000FEE7FEE7FEE7FEE74F190008250100085D
:1001700032490143324A1160704770B500210023B3
:100180000F22C4781CB32E4C246804F4E064C4F538
:10019000E064C4F30721C1F10404E3B20A414478E6
:1001A0009C40E1B28478144021430C07210E254C79
:1001B00005786155047804F01F050124AC400578EA
:1001C0006D11AD0005F1E025C5F8004109E00478A6
:1001D00004F01F050124AC401B4D0678761145F84C
:1001E000264070BD194A0A400243154B1B1F1A6076
:1001F000704739B1124A121D12680243104B1B1D81
:100200001A6006E00E4A121D126882430C4B1B1D39
:100210001A607047042808D14FF0E021096941F0C5
:1002200004014FF0E022116107E04FF0E02109697D
:1002300021F004014FF0E022116170470000FA053F
:100240000CED00E000E400E080E100E080FFFF1F33
:1002500001460020F94A106820F0010008431060B0
:10026000704730B1F549096841F00201F34A116065
:1002700005E0F249096821F00201F04A1160704777
:1002800030B1EE49096841F00401EC4A116005E023
:10029000EA49096821F00401E84A1160704730B169
:1002A000E649096841F00801E44A116005E0E349C4
:1002B000096821F00801E14A11607047DF48001D1C
:1002C000006800F0010028B1DD48DC490C3108600D
:1002D000DC480860704700B5D848001D006800F091
:1002E000020038B1FFF7EAFFD748D449103108605F
:1002F000D648086000BDD148001D006840F00200EB
:10030000CE49091D086070470420CC49183109689E
:1003100001F0010109B1012010E0C8491831096854
:1003200001F4807109B1022008E0C449183109685C
:1003300001F4F05109B1032000E00420704708B532
:10034000024604200090FFF7DFFF009003E0FFF774
:10035000DBFF0090521E9DF80000012801D1002A09
:10036000F5D10AB9052000909DF8000008BD30B510
:10037000044604256803FFF7E2FF0546042D1FD15C
:10038000AE48001D006840F40070AC49091D0860CB
:100390000846006840F008000860002020606803FC
:1003A000FFF7CDFF0546A548001D006820F00800B6
:1003B000A249091D08600846006820F40070086022
:1003C000284630BD70B504460D4604267003FFF77D
:1003D000B6FF0646042E04D125604003FFF7AFFFA9
:1003E0000646304670BD9548001D006840F001008B
:1003F0009249091D0860704740B19049091D09687C
:1004000041F480718D4A121D116007E08B49091D6E
:10041000096821F48071894A121D1160704730B556
:10042000044604256803FFF78AFF0546042D01D121
:1004300000202070284630BD30B5044604256803EE
:10044000FFF77DFF0546042D01D1002020802846BE
:1004500030BD30B5044604256803FFF770FF05463C
:10046000042D01D100202060284630BD70B504461F
:100470000D4604267003FFF762FF0646042E0CD1DA
:100480006E48001D006820F480706C49091D0860EA
:1004900025707003FFF753FF0646304670BD70B5F8
:1004A00004460D4604267003FFF749FF0646042E56
:1004B0000CD16248001D006820F480705F49091D5E
:1004C000086025807003FFF73AFF0646304670BD8E
:1004D00070B504460D4604267003FFF730FF06464C
:1004E000042E0CD15548001D006820F4807053493B
:1004F000091D086025607003FFF721FF064630469E
:1005000070BD70B504460D4604267003FFF717FF53
:100510000646042E04D125704003FFF710FF06465F
:10052000304670BD70B504460D4604267003FFF7D3
:1005300006FF0646042E04D125804003FFF7FFFE88
:100540000646304670BD70B504460D46042670035D
:10055000FFF7F5FE0646042E04D125604003FFF7A1
:10056000EEFE0646304670BD00B53448001D0068FA
:1005700000F0040038B1FFF7A1FE35482F491431CF
:1005800008603448086000BD2C48001D006840F039
:1005900004002A49091D086070472848001D0068AA
:1005A00040F480202549091D086070472DE9F04777
:1005B00004460F46002500264FF00408A946AA4627
:1005C0004FF40040FFF7BBFE8046B8F1040F31D175
:1005D000AFB121488068204385B21F48C06840EA17
:1005E000144086B2E84345EA00491B48C0F8089029
:1005F000F04346EA004A1848C0F80CA015E0164837
:10060000806880B220EA04051348C068E14300EA2C
:100610001146E84345EA00490F48C0F80890F04306
:1006200046EA004A0C48C0F80CA04FF40040FFF71F
:1006300086FE80464046BDE8F0870000003C024050
:10064000EFCDAB8905040302BFAE9D8C16151413C4
:10065000C8D9EAFB272625240000F81F2DE9F0471A
:1006600004460F46002500264FF00408A946AA4676
:100670004FF40040FFF763FE8046B8F1040F31D11C
:10068000AFB1A0480069204385B29E48406940EA66
:10069000144086B2E84345EA00499A48C0F81090F1
:1006A000F04346EA004A9748C0F814A015E0954880
:1006B000006980B220EA040592484069E14300EAFB
:1006C0001146E84345EA00498E48C0F81090F043CF
:1006D00046EA004A8B48C0F814A04FF40040FFF7E8
:1006E0002EFE80464046BDE8F0872DE9F0470446DF
:1006F0000F46002500264FF00408A946AA464FF4ED
:100700000040FFF71CFE8046B8F1040F31D1AFB1B5
:100710007C488069204385B27A48C06940EA144029
:1007200086B2E84345EA00497648C0F81890F0439D
:1007300046EA004A7348C0F81CA015E07148806979
:1007400080B220EA04056F48C069E14300EA11461F
:10075000E84345EA00496B48C0F81890F04346EA80
:10076000004A6848C0F81CA04FF40040FFF7E7FDBE
:1007700080464046BDE8F087F0B5044604250026D3
:1007800000276803FFF7DBFD0546E043C6B244EAF5
:100790000647042D01D15B4807604FF40040FFF786
:1007A000CEFD05462846F0BD2DE9F04304460D4632
:1007B000164604274FF000084FF000095248006821
:1007C000C0F3034944EA0500304340EA0900C0434E
:1007D0004FEA004844EA0500304340EA090040EA95
:1007E00008087803FFF7ABFD0746042F02D1454800
:1007F000C0F804804FF40040FFF7A1FD07463846DB
:10080000BDE8F083F0B504460425002600273E48E5
:10081000006800F47000070C44EA0700C0430604B7
:1008200044EA070006436803FFF789FD0546042DE7
:1008300001D1344846604FF40040FFF780FD054683
:100840002846F0BDF0B504460425002600272E48B2
:100850000068C0F3064744EA0700C043060444EAC0
:10086000070006436803FFF76AFD0546042D01D122
:10087000244846604FF40040FFF761FD05462846D6
:10088000F0BD21480068C0F3075070471E48001DA6
:10089000006870471C486430006870471A48683028
:1008A00000687047002018490968C9B2AA2901D018
:1008B000012000E00020704713480068C0F30340A7
:1008C000704739B1104A183A126802430E4B183B70
:1008D0001A6006E00C4A183A126882430A4B183B29
:1008E0001A60704701460020074A121F12680A402A
:1008F0000AB1012000E0002070470349091F086089
:10090000704700000000F81F1C3C024010B5044670
:100910008548844208D10121084600F0BCFA002134
:10092000012000F0B8FA52E08048844208D1012149
:10093000022000F0B0FA0021022000F0ACFA46E0FC
:100940007B48844208D10121042000F0A4FA002150
:10095000042000F0A0FA3AE07648844208D1012150
:10096000082000F098FA0021082000F094FA2EE008
:100970007148844208D10121102000F08CFA002136
:10098000102000F088FA22E06C48844208D101214E
:10099000402000F080FA0021402000F07CFA16E0B0
:1009A0006748844208D10121802000F074FA0021B8
:1009B000802000F070FA0AE06248844207D10121E9
:1009C000202000F068FA0021202000F064FA10BD19
:1009D000F0B50A4600210023002400BF3DE00125B8
:1009E00005FA01F3156805EA03049C4234D1056851
:1009F0004F000326BE40B543056015794E00B54053
:100A00000668354305601579012D02D01579022D50
:100A100016D185684F000326BE40B54385605579E1
:100A20004E00B540866835438560858801268E4036
:100A3000B5438580858896798E40B6B235438580EA
:100A4000C5684F000326BE40B543C560D5794E004A
:100A5000B540C6683543C560491C1029BFD3F0BDF9
:100A60004FF6FF7101600021017141718171C17107
:100A7000704708B54FF480320092009A0A43009202
:100A8000009AC261C161009AC261C2690092C269E2
:100A9000009208BD02460020138A0B400BB10120D2
:100AA00000E0002070470146088A70470246002097
:100AB000938A0B400BB1012000E0002070470146F3
:100AC000888A704701837047418370470AB1018368
:100AD00000E04183704781827047828A4A40828267
:100AE0007047F0B5002300244D07ED0E02FA05F320
:100AF000CE1000F1200555F826504E07F70E0F26B0
:100B0000BE40B543CF1000F1200646F82750CE1066
:100B100000F1200555F8265045EA0304CE1000F1F7
:100B2000200545F82640F0BD0000024000040240C8
:100B300000080240000C0240001002400018024071
:100B4000001C024000140240F948006840F4807024
:100B5000F7490860F64808300068F6490840F4494B
:100B600008310860F2480068F3490840F04908601D
:100B70000846006820F480200860ED4808300068CE
:100B800020F47D00EA49083108600020091D086052
:100B900070470021E64A921C117011460870704798
:100BA00010B501460022002300204A11012A02D17B
:100BB000DF4C236802E0DE4C3434236801F01F026E
:100BC000012494401C400CB1012000E0002010BD25
:100BD00038B5002000900024002500BF3120FFF729
:100BE000DFFF05460098401C00900098B0F5A06F0C
:100BF00001D0002DF2D03120FFF7D2FF08B101243F
:100C000000E00024204638BDC949C91D087070475E
:100C100001460020C64A121D106820F460400843B7
:100C200010607047C5490862704701460020C04AFD
:100C3000121D106820F4F85040EA0120106070473F
:100C4000BE49086070470021B94A3532117011461B
:100C500008707047BA490860704710B541EA02034E
:100C60000343B34C0A34237010BDB449086670477F
:100C7000B24908677047B2492C310860704740EAB2
:100C80000102AB4B0B331A70704701460020A84A93
:100C90000832106820F00300084310607047A44831
:100CA0000830006800F00C00704701460020A04AA0
:100CB0000832106820F0F0000843106070470146C9
:100CC00000209B4A0832106820F4E060084310605E
:100CD000704701460020964A0832106820F46050A0
:100CE00040EAC10010607047F0B5002100220023E7
:100CF0000026002400258E4F08373F6807F00C01BE
:100D000031B1042912D0082913D00C2937D113E0AE
:100D1000874F3F1D3F68C7F342356F1C4FF0010CF2
:100D20000CFA07FC4FEACC37076036E0854F0760C6
:100D300033E0854F076030E07D4F08373F6807F4A8
:100D400070127B4F08373F6807F440037F4F07EB73
:100D500092473A78012707EB9353754F08373F685E
:100D600007F480362EB9774F5743B7FBF3F7076088
:100D700004E0754F5743B7FBF3F707600DE06C4F86
:100D80003F1D3F68C7F342356F1C4FF0010C0CFA52
:100D900007FC4FEACC37076000BF00BF644F08373D
:100DA0003F6807F0F0010909694F7C5C0768E7407C
:100DB00047605F4F08373F6807F4E061090A644FF6
:100DC0007C5C4768E7408760594F08373F6807F405
:100DD0006051C90A5E4F7C5C4768E740C760F0BD60
:100DE000002100F44032B2F5403F08D1504A11686A
:100DF00021F0C04100F0C04211434D4A11604C4AFD
:100E00003432126822F44032494B34331A601A46A5
:100E1000126800F440331A43454B34331A6070476C
:100E2000474958310860704745495C310860704750
:100E300039B13F4A1C32126802433D4B1C331A60E1
:100E400006E03B4A1C3212688243394B1C331A605D
:100E5000704739B1364A203212680243344B20338E
:100E60001A6006E0324A203212688243304B203347
:100E70001A60704739B12E4A2432126802432C4B53
:100E800024331A6006E02A4A243212688243284B2F
:100E900024331A60704739B1254A10321268024370
:100EA000234B10331A6006E0214A10321268824345
:100EB0001F4B10331A60704739B11D4A1432126843
:100EC00002431B4B14331A6006E0194A14321268AD
:100ED0008243174B14331A60704739B1144A1832E1
:100EE00012680243124B18331A6006E0104A183297
:100EF000126882430E4B18331A60704739B10C4A9E
:100F00002832126802430A4B28331A6006E0084A66
:100F1000283212688243064B28331A607047C9B1E1
:100F2000034A2C3212680243014B2C331A6016E03C
:100F3000003802400CC0FF88FEFFFEEE0000474272
:100F4000800647420024F40000127A0000000020CE
:100F5000090000201F4A126882431E4B1A60704726
:100F600039B11C4A121D126802431A4B1B1D1A602C
:100F700006E0184A121D12688243164B1B1D1A60A8
:100F8000704739B1134A1F3A12780243114B1F3B85
:100F90001A7006E00F4A1F3A127882430D4B1F3B2E
:100FA0001A7070470B480830006840F0807009499B
:100FB00008310860704701460020064A203A12684E
:100FC0000A400AB1012000E00020704701491E39A3
:100FD000087070472C38024010B50446BA48844265
:100FE00008D101218014FFF767FF0021A014FFF74B
:100FF00063FF16E0B548844208D101210014FFF7D1
:101000006CFF00212014FFF768FF0AE0B04884421B
:1010100007D10121C013FFF760FF0021E013FFF7A4
:101020005CFF10BD10B50022028802F441520B880B
:101030004C8823438C882343CC8823430C89234347
:101040004C8923438C892343CC8923431A43028050
:10105000838B4FF2FF74234083830B8A038210BD7E
:101060002DE9FF5F05460C464FF0000902274FF0BF
:1010700000084FF0010B0026B246A88B4FF240014A
:101080000840A88302202884B5F81C90A068022894
:1010900001D100BF33E0A08810B94FF0010B01E08F
:1010A0004FF0020B6846FFF71FFEDDF800A0E08856
:1010B000B0F5007F0AD14FEA1A2000EB8000400013
:1010C000A168B0FBF1F0401D86B20BE04FEA4B1077
:1010D000BAFBF0F000EB80004000A168B0FBF1F03B
:1010E000401D86B20A20B6FBF0F606F00108A6EB1A
:1010F0000800C0F34F074FF6FF7000EA0828022FE0
:1011000001DBFF2F02DD02274FF00008E08840EAF4
:10111000080038432884A088A189084361880843CF
:101120002188084340F4006040EA0909A5F81C90B2
:10113000BDE8FF9F0021018041808180C180018145
:1011400041818181C1810721018270470021018095
:1011500041808180C18002218160002181817047AE
:1011600021B1028842F04002028004E002884FF67A
:10117000BF731A400280704721B1828B42F48062B3
:10118000828304E0828B4FF6FF331A4082837047DC
:1011900002884FF2FF731A40028002880A430280DD
:1011A0007047B1F5804F04D1028842F4804202803A
:1011B00004E002884BF6FF731A40028070474FF636
:1011C000FF62914204D0028842F48072028004E0FF
:1011D00002884FF6FF631A400280704721B182886F
:1011E00042F00402828004E082884FF6FB731A40CA
:1011F000828070470146888970478181704721B19C
:10120000028842F40052028004E002884DF6FF7327
:101210001A4002807047018841F480510180704774
:1012200002460020012901D0108B00E0908A70470F
:101230000146088A70471AB183880B43838002E015
:1012400083888B438380704730B5002400230C11C2
:101250000125A540ABB21AB185881D43858002E007
:1012600085889D43858030BD0246002013890B4050
:101270000BB1012000E000207047CA430281704793
:10128000F0B50246002000240023002501F00F07DE
:101290000126BE40B4B20B1101269E40B3B296881F
:1012A00006EA03051689264016B10DB1012000E0BB
:1012B0000020F0BD10B5002201F00F040123A3406F
:1012C0009AB2D343038110BD003001400038004082
:1012D000003C004010B50446F748844209D1012182
:1012E0008803FFF7E9FD00214FF48040FFF7E4FD9C
:1012F00032E0F248844209D101214804FFF7EDFDB4
:1013000000214FF40030FFF7E8FD25E0EC4884426F
:1013100009D101218804FFF7E0FD00214FF480206E
:10132000FFF7DBFD18E0E748844209D10121C8043A
:10133000FFF7D3FD00214FF40020FFF7CEFD0BE0B7
:10134000E148844208D101210805FFF7C6FD0021CC
:101350004FF48010FFF7C1FD10BD2DE9FF47054692
:101360000E460024A14600BFA046B08900B100BFD0
:101370002C8A24F44054F08804432C82AC8941F236
:101380000C608443B0883189084371890843044361
:10139000AC81AC8A24F44074B0890443AC826846C2
:1013A000FFF7A2FCC448854202D1DDF80C9001E0B1
:1013B000DDF80890A88900F4004040B109EBC900AD
:1013C00000EB091031684900B0FBF1F707E009EBC9
:1013D000C90000EB091031688900B0FBF1F7642007
:1013E000B7FBF0F004012009642101FB1078A88903
:1013F00000F4004040B1322000EBC800B0FBF1F037
:1014000000F00700044308E0322000EB08106421DC
:10141000B0FBF1F000F00F0004432C81BDE8FF8722
:101420004FF41651016000218180C18001810C219F
:10143000418100218181704710B502460020108A49
:1014400020F470600B884C8823438C882343CC881D
:1014500023431843108210BD002101804180818008
:10146000C180704721B1828942F40052828104E038
:1014700082894DF6FF731A4082817047028B02F415
:101480007F420283028B0A430283704721B1828923
:1014900042F40042828103E08289C2F30E0282811B
:1014A000704721B1828A42F40062828204E0828A1B
:1014B0004FF2FF731A4082827047C1F308028280A4
:1014C000704701468888C0F308007047028A4FF6CB
:1014D000F0731A400282028A0A430282704721B1E5
:1014E000828942F00202828104E082894FF6FD7314
:1014F0001A408281704782894FF2FF731A408281BD
:1015000082890A4382817047028A4FF6DF731A404C
:101510000282028A0A430282704721B1028A42F49F
:101520008042028204E0028A4BF6FF731A40028274
:101530007047818941F001018181704721B1828A20
:1015400042F00802828204E0828A4FF6F7731A4062
:1015500082827047028BD2B20283028B42EA01225E
:101560000283704721B1828A42F02002828204E025
:10157000828A4FF6DF731A408282704721B1828AD5
:1015800042F01002828204E0828A4FF6EF731A4022
:1015900082827047828A4FF6FB731A408282828A67
:1015A0000A438282704721B1828A42F0020282821B
:1015B00004E0828A4FF6FD731A40828270471AB1A6
:1015C000838A0B43838202E0838A8B438382704742
:1015D000F0B50346002400260025002040F66A17D7
:1015E000B94200D100BF1846C1F3421401F01F06F2
:1015F000012707FA06F5012C01D10C3004E0022C7A
:1016000001D1103000E014301AB107682F43076091
:1016100002E00768AF430760F0BD02460020B1F565
:10162000007F00D100BF13880B400BB1012000E008
:101630000020704701F40072B2F5007F00D100BFB6
:10164000CA430280704770B502460024002300257B
:10165000002040F66A16B14200D100BFC1F3421526
:1016600001F01F03012606FA03F3012D02D196892A
:10167000334006E0022D02D1168A334001E0968AFB
:1016800033400C12012606FA04F41688344013B1D4
:101690000CB1012000E0002070BD10B50022002335
:1016A00040F66A14A14200D100BF0A1201249440FE
:1016B000A3B2DC43048010BD003801400044004068
:1016C00000480040004C00400050004008B5002495
:1016D00000250020009000F041FA4CE031208DF808
:1016E000000025A001F0A7F80446B4F57A7F3CD9A4
:1016F00072B6214622A000F050FE012000EB142516
:1017000024A000F04AFEA9B2284800F0CBFE28A091
:1017100000F043FE2BA000F040FE2246002116A060
:1017200001F0ACF82EA000F038FE13A001F067F82D
:101730002FA000F032FEFEF7C1FD3448FEF76FFE29
:10174000FEF751FEFEF7BAFD31213048FEF78EFE5E
:10175000FEF749FE9DF800102DA000F01EFE31A0FE
:1017600000F01BFE114803F0E1FE32A000F015FE70
:101770000E4803F0DBFEB1E74150502E62696E0067
:101780004150502053697A652069733A256C640D85
:101790000A00000073747261742065726173652EB3
:1017A0002E2E2E2E2E2E2E0D0A00000000000108D7
:1017B000656E642065726173652E2E2E2E2E2E2E80
:1017C0002E0D0A0072656164203C3C4150502E622F
:1017D000696E3E3E2E2E2E2E2E2E2E2E0D0A00002F
:1017E0007265616420656E642E2E2E2E2E0D0A0009
:1017F0006961705F6C6F61645F61707020737563A5
:101800006573732121210D0A00000000BC00080847
:101810004941505F466C6167206973203A25780D15
:101820000A0000006A756D7020746F206170700D81
:101830000A000000415050206973206E6F742066CA
:10184000696E6421212121210D0A00000CB50020C0
:10185000019000908748006840F480308549086016
:1018600000BF8448006800F4003000900198401CDC
:101870000190009818B90198B0F5A06FF1D17D489A
:10188000006800F4003010B10120009001E0002059
:1018900000900098012859D17748006840F0040072
:1018A000754908600846006840F002000860084674
:1018B000006840F0010008606E482430006840F085
:1018C00080506C4924310860C8146C49086000BF1E
:1018D0006A48406800F010000028F9D165480830D7
:1018E00000686449083108600846006808600846D6
:1018F000006808600846006820F47D00086008461B
:10190000006840F49A0008605A48006840F080700F
:101910005849086000BF5748006800F00070002870
:10192000F9D054480830006820F0030051490831CC
:1019300008600846006840F00300086000BF4D489A
:101940000830006800F00C000C28F8D10CBD10B570
:101950004848006840F480704649086045480830AF
:101960000068474908404349083108604148006819
:10197000444908403F4908600846006820F4802038
:1019800008603C480830006820F47D00394908317F
:1019900008600020091D0860FFF758FF4FF0006045
:1019A0003949086010BD70B50022002000210024D4
:1019B0000023304D08352D6805F00C0232B1042AA1
:1019C00010D0082A12D00C2A39D113E0294D2D1D30
:1019D0002D68C5F342335D1C0126AE40F5032B4E46
:1019E000356038E02A4D294E356034E0294D274EC8
:1019F000356030E01F4D08352D6805F470101D4D21
:101A000008352D6805F44001234D05EB90452878F5
:101A1000012505EB9151174D08352D6805F48034EB
:101A200034B91B4D4543B5FBF1F5184E356005E063
:101A3000184D4543B5FBF1F5144E35600BE00D4DE7
:101A40002D1D2D68C5F342335D1C0126AE40F50304
:101A50000E4E356000BF00BF064D08352D68C5F33A
:101A600003150E4E725D094D2D68D540074E356049
:101A700070BD000000380240003C02400070004091
:101A80000CC0FF88FEFFFEEE08ED00E01C00002009
:101A90000024F40000127A00200000202900002019
:101AA000704710E000BFBFF34F8F0B48006800F491
:101AB000E0600A490843001D07490860BFF34F8FE3
:101AC00000BF00BFFEE7EDE700BFFEE700BFFEE797
:101AD00000BFFEE7704700000CED00E00000FA05D3
:101AE0001A48006840F080701849086000201849C2
:101AF00048600846006840F001000860704730B553
:101B0000134C63680021134C2468134DB4FBF5F4A7
:101B100004FB00F202E00E4C6468E11A9142FAD331
:101B200030BD10B504464FF47A7104FB01F0FFF7A5
:101B3000E6FF10BD10B500210246054C636802E0C7
:101B4000034C6468E11A9142FAD310BDFCED00E049
:101B5000001000E01C00002040420F0010B54FF4C0
:101B60004070FEF705FBFFF7BBFF00F00BF81021FC
:101B70000348FEF7A7FF4FF4165000F053FB10BDCB
:101B8000000002401CB501210846FFF751F9102062
:101B9000009001208DF8040000208DF8060001203F
:101BA0008DF8070000208DF8050069460648FEF70D
:101BB0000FFF4FF480510448FEF786FF10210248C2
:101BC000FEF782FF1CBD00000000024000B587B098
:101BD00001210620FFF72CF901208DF818000020C4
:101BE0008DF81A0001208DF81B0002208DF81900D5
:101BF0004020059005A94948FEF7EAFE40214748E4
:101C0000FEF760FF02208DF8180000208DF81A0002
:101C100002208DF819004FF46040059005A9404856
:101C2000FEF7D6FE4FF460413D48FEF74BFF05221C
:101C30000D213B48FEF755FF05220E213848FEF7DF
:101C400050FF05220F213648FEF74BFF0121880384
:101C5000FFF710F90020ADF800004FF48270ADF8E6
:101C600002000020ADF80400ADF80600ADF8080051
:101C70004FF40070ADF80A001020ADF80C00002001
:101C8000ADF80E000720ADF8100069462548FFF7B3
:101C9000C9F901212348FFF763FA07B000BD00F03E
:101CA0000700204909884FF6C77211401D4A11806C
:101CB0001146098841EAC00111801146098841F0A6
:101CC0004001118070470246002107E0481C81B2A4
:101CD0004FF6FE70814201DB00207047114808304A
:101CE000008800F002000028F0D00E480C3002807E
:101CF000002107E0481C81B24FF6FE70814201DBF3
:101D00000020EAE707480830008800F001000028BA
:101D1000F0D004480C300088C0B2DEE70008024072
:101D2000000402400038004010B504462046FFF78A
:101D3000CAFF10BD10B53820FFF7B1FF10BD10B5B8
:101D40000020FFF7ACFF10BD10B5FFF73FFF0720E5
:101D5000FFF7A5FF10BD10B54021FC48FEF7B2FE0D
:101D6000FF20FFF7E1FF10BD10B5002400BFFF20EA
:101D7000FFF7DAFFFF2801D1002010BD641C6FF0CF
:101D80007F408442F3D30120F7E710B54021EF48AC
:101D9000FEF79AFEFFF7E8FF08B9002010BDFFF735
:101DA000DAFF0120FAE770B505464FF6FF7401E04F
:101DB000601E84B2FF20FFF7B7FFA84201D0002CBD
:101DC000F6D10CB9FF2070BD0020FCE770B50446C9
:101DD0000D46FE20FFF7E7FF08B1012070BD04E0CB
:101DE000FF20FFF770FF2070641C281EA5F1010181
:101DF0008DB2F5D1FF20FFF797FFFF20FFF794FF8B
:101E00000020EBE770B506460D46FFF7ADFF08B1C1
:101E1000012070BD2846FFF787FFFD2D19D0002453
:101E200004E0305DFFF74FFF601C84B2B4F5007F23
:101E3000F7DBFF20FFF778FFFF20FFF775FFFF209C
:101E4000FFF772FF044604F01F00052801D00220AE
:101E5000DFE70020DDE72DE9F04105460C46174697
:101E60004FF00008FFF777FFFFF78FFF10B1FF205B
:101E7000BDE8F08145F04000FFF756FF200EFFF768
:101E800053FFC4F30740FFF74FFFC4F30720FFF7EA
:101E90004BFFE0B2FFF748FF3846FFF745FF0C2D38
:101EA00002D1FF20FFF740FF4FF01F0800BFFF20C7
:101EB000FFF73AFF064606F0800030B1B8F10000A7
:101EC000A8F1010101F0FF08F1D13046D0E770B56B
:101ED0000546012200210A20FFF7BDFF044624B970
:101EE00010212846FFF772FF0446FFF734FF0CB1BC
:101EF000012070BD0020FCE770B5054601220021DD
:101F00000920FFF7A8FF044624B910212846FFF74F
:101F10005DFF0446FFF71FFF0CB1012070BD0020DC
:101F2000FCE77FB56846FFF7E7FF10B1002004B07B
:101F300070BD9DF8000000F0C000402809D19DF858
:101F400009009DF8081000EB0120401C84B2A50296
:101F500020E09DF8050000F00F009DF80A1000EB4E
:101F6000D1109DF8091001F0030100EB4100861C1F
:101F70009DF8080080119DF8071000EB81009DF886
:101F8000061001F0030100EB8120441CA6F10900BA
:101F900004FA00F52846CAE7F8B5FFF7D5FEFFF7C3
:101FA000C9FE002504E0FF20FFF7BEFE681C85B2D5
:101FB0000A2DF8DB142600BF952200210846FFF702
:101FC0004AFF0446012C04D0301EA6F101018EB256
:101FD000F2D100205E490870012C4AD187224FF4CB
:101FE000D5710820FFF737FF012847D1002506E00B
:101FF000FF20FFF799FE0DF80500681C85B2042D3F
:10200000F6DB9DF80200012879D19DF80300AA288B
:1020100075D14FF6FE7600BF012200213720FFF771
:102020001AFF012291072920FFF715FF044624B16A
:10203000301EA6F101018EB2EED1002E5FD001223A
:1020400000213A20FFF707FF002858D1002506E0BD
:10205000FF20FFF769FE0DF80500681C85B2042D0E
:10206000F6DB9DF8000000F0400018B1062038496A
:10207000087044E004203649087040E00122002145
:102080003720FFF7E8FE012200212920FFF7E3FEB9
:102090000446012C17DC02202D4908704FF6FE760D
:1020A00000BF012200213720FFF7D5FE01220021C9
:1020B0002920FFF7D0FE0446BCB1301EA6F1010175
:1020C0008EB2EED111E00120214908704FF6FE7664
:1020D00000BF012200211046FFF7BDFE044624B1D7
:1020E000301EA6F101018EB2F3D12EB101225102B0
:1020F0001020FFF7B0FE10B1002015490870FFF75F
:102100002AFEFFF71CFE1248007808B10020F8BD37
:102110000CB12046FBE7AA20F9E72DE9F04106467D
:102120000F4615460A480078062800D07F02012D88
:1021300010D1012239461120FFF78DFE04461CBB49
:1021400069023046FFF742FE04461DE000080240E7
:1021500039000020012239461220FFF77CFE044698
:1021600000BF4FF400713046FFF730FE044606F51D
:102170000076681EC0B2051E01D0002CF1D00122ED
:1021800000210C20FFF767FEFFF7E5FD2046BDE8C4
:10219000F0812DE9F04106460F46154620480078AB
:1021A000062800D07F02012D0CD1012239461820CB
:1021B000FFF751FE04466CBBFE213046FFF722FEBE
:1021C000044627E016480078012809D001220021A2
:1021D0003720FFF740FE012229461720FFF73BFE7C
:1021E000012239461920FFF736FE044694B900BF94
:1021F000FC213046FFF706FE044606F50076681E11
:10220000C0B2051E01D0002CF2D0FD210020FFF746
:10221000F9FD0446FFF79FFD2046BDE8F081000070
:102220003900002010B588B0044601210805FEF7EA
:1022300021FE01210C20FEF7FBFD6A48FFF74AF85A
:102240004FF48050029002208DF80C008DF80D00A4
:1022500000208DF80E0001208DF80F0002A96248C1
:10226000FEF7B6FB0420029002208DF80C008DF8DA
:102270000D0000208DF80E0001208DF80F0002A93E
:102280005A48FEF7A5FB08220C215748FEF729FC07
:10229000082202215548FEF724FC04940020ADF8E2
:1022A0001400ADF81600ADF81800ADF81C000C20B5
:1022B000ADF81A0004A94B48FFF74FF8012149482F
:1022C000FFF7D0F8012240F225514648FFF780F988
:1022D00031208DF8040003208DF8050000208DF8D2
:1022E000060001208DF8070001A8FDF746FF4021F8
:1022F0003C48FFF79FF908B010BD10B53C48B0F856
:1023000064006FF30E003A49A1F864000846B0F883
:10231000640020F40040A1F864006421344803F014
:1023200024F9C821334803F020F910BD10B540F25C
:1023300025512C48FFF787F9C8B12A48FFF7C1F8A3
:10234000C4B22B48B0F86400C0F30E0063280EDA64
:102350002749B1F86410C1F30E00411C244AB2F8B9
:10236000642061F30E022249A1F864200C5440F26B
:1023700024411C48FFF767F901280DD11C48B0F82B
:10238000640020F4004000F500401949A1F8640001
:102390001448FFF796F8C4B210BD0FB438B505A8BD
:1023A00000901448009A049903F0A4FB00200090C8
:1023B000104803F0E5F885B200240DE000BF40218D
:1023C0000848FFF72AF90028F9D00A48015D0548B6
:1023D000FFF773F8601C84B2AC42EFDB38BC5DF8E9
:1023E00014FB00000050004000080240000C0240B6
:1023F00058000020BE00002001460878704730B524
:1024000003460C461546002205E01846FFF7F4FF88
:10241000A0545B1C521CAA42F7D330BD2DE9F041F9
:1024200005460E461746B5F1006F01D2BDE8F081B2
:10243000FDF751FF41F60270FEF75FFA002406E057
:1024400028193168FDF7BEFF361D201D84B2BC423D
:10245000F6D3FDF750FF00BFE8E72DE9F041044651
:102460000D46B4F5007F01DDBDE8F0811C4800EBAE
:102470000426FDF730FF41F60270FEF73EFA3046C3
:10248000FDF775FF002707E030462968FDF79AFF42
:10249000361D2D1D381D87B2FF2FF5DDFDF72BFFF3
:1024A00000BFE1E72DE9F04105460E46B5F5007F96
:1024B00001D9BDE8F081FDF70EFF41F60270FEF78D
:1024C0001CFA002406E005EB04273846FDF74FFF11
:1024D000601C84B2B442F6DBFDF70DFF00BFE8E7F5
:1024E0000000010870B504460D4629462046FEF757
:1024F000E4FF00BF40212046FFF78FF80028F9D005
:1025000070BD70B505460C4604E021782846FFF7FB
:10251000E9FF641C20780028F7D170BD2DE9F04157
:1025200007460D46164600240CE0295D3846FEF7A6
:10253000C4FF00BF40213846FFF76FF80028F9D0EC
:10254000601C84B2B442F0DBBDE8F08170B5044693
:102550000D4640216C48FFF76DF8E1B26A48FEF77E
:10256000ACFF00BF80216848FFF757F80028F9D07A
:10257000204670BD10B588B0044601218803FEF7DF
:1025800068FC01210846FEF753FC5F48FEF7A2FEF7
:102590004FF4C060029002208DF80C008DF80D0001
:1025A00000208DF80E0001208DF80F0002A9574879
:1025B000FEF70EFA4FF48060029002A95348FEF72E
:1025C00007FA072209215148FEF78BFA07220A2150
:1025D0004E48FEF786FA04940020ADF81400ADF8DA
:1025E0001600ADF81800ADF81C000C20ADF81A006C
:1025F00004A94548FEF7B1FE012240F225514248A8
:10260000FEF7E6FF25208DF8040003208DF8050075
:1026100000208DF8060001208DF8070001A8FDF7C5
:10262000ACFD01213848FEF71DFF40213648FFF779
:1026300001F808B010BD1CB500213348FEF712FFA9
:102640003148FEF747FE01210846FEF7F1FB4FF443
:10265000C060009001208DF8040000208DF8060075
:1026600001208DF8070000208DF8050069462748F5
:10267000FEF7AEF94FF400712448FEF723FA4FF449
:1026800080612248FEF71EFA1CBD1CB500211E48C1
:10269000FEF7E8FE1C48FEF71DFE01210220FEF7B2
:1026A000C7FBC020009001208DF8040000208DF8A9
:1026B000060001208DF8070000208DF8050069460E
:1026C0001348FEF785F940211148FEF7FBF98021F8
:1026D0000F48FEF7F7F91CBD10B540F225510A4826
:1026E000FEF7B1FF70B10848FEF7EBFEC4B2214619
:1026F0000548FEF7E2FE00BF40210348FEF78DFFCC
:102700000028F9D010BD0000003801400000024050
:102710000004024070B586B004460D46164696A3E6
:10272000224697A1684603F0D1F99749002001F0AD
:10273000FDF813222146954801F00BF99348C16832
:1027400001F067FC05AB32462946904801F0AFFA2C
:102750008E4801F018FC0021084601F0E7F806B0A9
:1027600070BDFEB5002400200090019002908649C3
:1027700001F0DCF813226946844801F0EAF80546C6
:1027800025B300BF12E0601CC4B2804801F0FBFB1F
:102790000021084601F0CAF87B49002001F0C6F884
:1027A00013226946794801F0D4F805460DB101209D
:1027B00000E00020642C01DA012100E00021084043
:1027C0000028E0D1622C01DD0520FEBD6F48C16804
:1027D00001F01FFC6E4802F0D3FE06466D4B3246F8
:1027E0006B496A4801F063FA6A4B02226AA16748A2
:1027F00001F05DFA654801F0C6FB0020E5E73EB553
:1028000004460020009001900290224663A1684691
:1028100003F05CF95C49002001F088F8684601F09B
:10282000C2FE0546594801F0AEFB0021084601F002
:102830007DF828463EBD70B586B004464EA32246BC
:102840004FA101A803F042F94F49002001F06EF8B2
:102850000646012252A14D4801F07BF8064616B10A
:10286000042006B070BD4948C56801F08CFB0646DF
:102870000021084601F05AF82846F2E72DE9F04F0A
:10288000ADF5017D0646884614464FEA542AC4F346
:10289000080B4FF40171684602F067FE3A490020C8
:1028A00001F044F8814601223146384801F051F8E0
:1028B0008146002710E0354801F065FB814632492A
:1028C000002001F033F88146012231462F4801F003
:1028D00040F88146781CC7B2B9F1000F01D0012041
:1028E00000E00020642F01DA012100E0002108400F
:1028F0000028E0D14146254801F08BFB002508E087
:10290000244B4FF400726946204801F0D9F8814603
:102910006D1C5545F4D34FF40171684602F025FE55
:102920001C4B5A466946194801F0CAF8174801F08D
:102930002AFB81460021084600F0F8FF0DF5017DD5
:10294000BDE8F08F0EB51049002000F0EFFF012226
:1029500015A10E4800F0FDFF0E4B0A2269460B48F8
:1029600001F0AEF8019800F07F40B0F1006F01D1A6
:1029700000200EBD0120FCE72E74787400000000DA
:1029800025732573000000009C08002074060020B9
:10299000C8020020400000200D0A0000257300003E
:1029A0004150502E62696E004141502E62696E00A6
:1029B00070B503460C4603E014F8015B03F8015BB5
:1029C000151EA2F10102F7D170BD30B5034601E03A
:1029D00003F8011B141EA2F10102F9D130BDF0B5BC
:1029E00003461C460D46002000BF161EA2F1010240
:1029F00007D014F8017B15F801CBA7EB0C06301EAD
:102A0000F3D0F0BD024600E0521C107810B11078EF
:102A10008842F9D1107870472DE9F04104460D46FF
:102A2000266BAE422FD0207908B36078012332465E
:102A300004F1340102F0F8FC10B10120BDE8F0818E
:102A400000202071D4E908100844B0420FD9E7787B
:102A50000AE0206A064460780123324604F134011A
:102A600002F0E2FC781EC7B2012FF2DC00BF55B1C4
:102A7000607801232A4604F1340102F09EFC08B17B
:102A80000120DBE725630020D8E770B5044600216C
:102A90002046FFF7C1FF0546002D59D120780328B5
:102AA0004FD1607900284CD0002020634FF4007291
:102AB000002104F13400FFF788FF552184F8321219
:102AC000AA2184F83312522084F834005221352090
:102AD00001556121362001554121372001557221D0
:102AE00084F8181284F81912412184F81A1261210D
:102AF00084F81B12217C84F81C12208A010A84F8B5
:102B00001D122069010C84F81E122069010E84F840
:102B10001F12217B84F82012A089010A84F8211257
:102B2000E068010C84F82212E068010E84F8231298
:102B30006078012304F13401626902F075FC002021
:102B4000607160780022114602F09BFC00B1012503
:102B5000284670BD0246891ED069801E884201D871
:102B6000002070479378D06A01FB0300F9E72DE954
:102B7000F04105460C46022C02D3E869A04202D877
:102B80000120BDE8F0812878012804D002282CD04B
:102B900003285AD13DE0274607EB5707686A00EB48
:102BA00057212846FFF738FF00B14EE0C7F3080170
:102BB00005F1340010F801807F1C686A00EB572192
:102BC0002846FFF729FF00B13FE0C7F3080105F1F0
:102BD0003400405C48EA002804F0010010B14FEADC
:102BE0001810CEE7C8F30B00CBE7686A00EB14219E
:102BF0002846FFF711FF00B127E040F2FF1000EA7E
:102C0000440105F134000E183078717840EA012053
:102C1000B7E7686A00EBD4112846FFF7FDFE00B164
:102C200013E040F2FF1000EA840105F134000E18B1
:102C3000F0780006B17840EA0140717840EA01205E
:102C40003178084320F070409BE700BF4FF0FF3021
:102C500097E72DE9F04705460E461746022E02D3A8
:102C6000E869B04202D84FF002088AE028780128CB
:102C700004D0022841D003287DD154E0B14609EBAD
:102C80005909686A00EB59212846FFF7C5FE8046BE
:102C9000B8F1000F00D071E0C9F3080105F134006C
:102CA0000C1806F0010020B1F9B2207861F31F1072
:102CB00000E03846207009F1010901202871686A96
:102CC00000EB59212846FFF7A7FE8046B8F1000F18
:102CD00000D053E0C9F3080105F134000C1806F0E8
:102CE000010010B1C7F3071005E0207800F0F000F4
:102CF000C7F303210843207040E0686A00EB162107
:102D00002846FFF789FE8046B8F1000F00D035E075
:102D100040F2FF1000EA460105F134000C1827705C
:102D2000380A60702AE0686A00EBD6112846FFF77F
:102D300073FE8046B8F1000F00D01FE040F2FF1094
:102D400000EA860105F134000C18E0780006A1784D
:102D500040EA0140617840EA01202178084300F010
:102D6000704007432770380A6070380CA070380E26
:102D7000E07003E0FFE74FF0020800BF00BF012052
:102D800028714046BDE8F0872DE9F04104460E4623
:102D9000022E02D3E069B04201D8022725E00027C5
:102DA0001FE031462046FFF7E2FE054605B91BE06D
:102DB000012D01D1022717E0681C08B9012713E093
:102DC000002231462046FFF744FF074607B10BE0DB
:102DD0002069401C20B12069401C206101206071E5
:102DE0002E46E069B042DCD800BF3846BDE8F0812D
:102DF0002DE9F04704468946B9F1000F06D1E7688E
:102E000017B1E069B84211D801270FE049462046C2
:102E1000FFF7ADFE0646022E02D20120BDE8F08784
:102E2000E069B04201D93046F8E74F463D4600BF61
:102E30006D1CE069A84204D80225BD4201D90020DA
:102E4000ECE729462046FFF792FE064606B909E060
:102E5000701C08B1012E01D13046DFE7BD42E7D139
:102E60000020DBE700BF6FF0704229462046FFF7E5
:102E7000F0FE8046B8F1000F08D1B9F1000F05D07F
:102E80002A4649462046FFF7E4FE8046B8F1000F87
:102E900009D1E5602069401C68B12069401E2061AD
:102EA0000120607107E0B8F1010F02D14FF0FF304F
:102EB00000E0012005462846B0E770B503460D4600
:102EC000586A021D680A1E68B678B0FBF6F400BFA7
:102ED00002CA09B9002070BD8C4200D202E0641A17
:102EE000121DF5E700BF10682044F4E72DE9F0411A
:102EF00004460E46E680A568012D03D02068C0690F
:102F0000A84202D80220BDE8F0812DB920680078DF
:102F1000032801D12068856A65B9E56020680089C9
:102F2000B04201DC0220EEE72068806A00EB161058
:102F3000206120E020688078070112E0294620689F
:102F4000FFF715FE0546681C08B90120DBE7022DD6
:102F500003D32068C069A84201D80220D3E7F01B40
:102F600086B2BE42EADAE56029462068FFF7F2FD44
:102F700000EB161020612068343006F00F0100EBE2
:102F8000411060610020BEE72DE9F041044688460B
:102F900000BFE088401C86B20EB1206910B9042041
:102FA000BDE8F08106F00F0000286FD12069401CB9
:102FB0002061E06828B920680089B04266DC0420FE
:102FC000EEE720688078401E00EA161000285DD1E8
:102FD000E1682068FFF7CBFD0546012D01D80220EE
:102FE000DEE7681C08B90120DAE72068C069A8425A
:102FF00046D8B8F1000F01D10420D1E7E16820687C
:10300000FFF7F6FE05460DB90720C9E7012D01D1EE
:103010000220C5E7681C08B90120C1E7002120682B
:10302000FFF7FAFC08B10120BAE7216801F134008A
:103030004FF400720021FFF7C8FC29462068FFF713
:1030400089FD21680863002710E0012021680871CC
:1030500000212068FFF7E0FC08B10120A0E720680C
:10306000006B401C21680863781CC7B22068807818
:10307000B842EADC2068006BC01B2168086300BF0F
:10308000E56029462068FFF765FD2061E68020683D
:10309000343006F00F0100EB4110606100207FE743
:1030A0002DE9F041044600212046FFF71FFF0546A9
:1030B00015B12846BDE8F08100BF21692068FFF7FF
:1030C000ABFC054605B116E0666937780FB90425F3
:1030D00011E0F07A00F0080030B90B223046A16907
:1030E000FFF77DFC00B906E000212046FFF74CFF0A
:1030F0000546002DE1D000BF2846DBE72DE9F04171
:10310000044604251AE021692068FFF785FC05467E
:1031100005B116E067693E780EB9042511E0E52E89
:1031200005D000BFF87A00F0080000B909E00021DE
:103130002046FFF729FF054605B102E02069002877
:10314000E1D100BF0DB1002020612846BDE8F0812B
:103150002DE9F041044600212046FFF7C7FE054651
:10316000ADB900BF21692068FFF756FC054605B1DF
:103170000CE060690678E52E00D006B906E0012172
:103180002046FFF701FF0546002DEBD000BF9DB99B
:1031900021692068FFF740FC05466DB96769202268
:1031A00000213846FFF711FC0B223846A169FFF7D2
:1031B000FFFB0120216808712846BDE8F08170B549
:1031C0000446E1882046FFF791FE05465DB9216976
:1031D0002068FFF721FC05462DB9E52061690870DC
:1031E000012021680871284670BD2DE9F35F019820
:1031F000D0F8008001E008F1010898F800002F28BD
:10320000F9D098F800005C28F5D0009885690B2269
:1032100020212846FFF7D9FB00263746B1464FF05C
:10322000080B18F809002E2825D100BF484609F1DF
:10323000010918F800402E2C02D1B9F1030F00D378
:1032400003E038467F1C2C54F0E700BF2F2C06D03B
:103250005C2C04D0202C02DD0620BDE8FC9F08EB8E
:10326000090101980160202C01DC242000E02020CD
:10327000E8720020F1E700BF484609F1010918F89B
:103280000040202C03DD2F2C01D05C2C00D152E01B
:103290002E2C01D05F450CD3BBF1080F01D12E2C91
:1032A00001D00620D9E708274FF00B0BB006060E19
:1032B000E2E7802C01DB46F00306812C20DBFE2CAC
:1032C0001EDC484609F1010918F800A0BAF1400FC8
:1032D00002DBBAF17E0F05DDBAF1800F06DBBAF131
:1032E000FE0F03DCABF10100B84201D80620B4E7C1
:1032F00038467F1C2C5438467F1C05F800A019E086
:103300002146FCA0FFF77EFB08B10620A5E7412C73
:1033100004DB5A2C02DC46F0020608E0612C06DBD6
:103320007A2C04DC46F00106A4F12000C4B2384631
:103330007F1C2C54A0E700BF08EB09010198016035
:10334000202C01DC042000E0002004460FB90620F8
:1033500083E72878E52801D105202870BBF1080F04
:1033600001D1B006060E06F00300012801D144F099
:10337000100406F00C00042801D144F00804EC729B
:1033800000206AE7F0B505460B4603F109022F69F4
:10339000002F40D06869067B00210AE0445C202CA5
:1033A00000D108E0052C00D1E52400BF02F8014B54
:1033B000491C0829F2D300BF077A202F0FD02E27EF
:1033C00002F8017B082107E0445C202C00D105E0D5
:1033D00000BF02F8014B491C0B29F5D300BFC77A87
:1033E0001F72C77F4FEA076C877F4CEA074C477F05
:1033F0004CEA072790F81CC047EA0C071F6090F8BA
:1034000018C0477E4CEA07279F8090F816C0C77DFA
:103410004CEA0727DF8000271770F0BD2DE9F34144
:103420000446019800782F2803D0019800785C2882
:1034300005D10198401C01900020A06002E02068A6
:103440008069A06001980078202807D200212046DA
:10345000FFF74CFD07460020606139E000BF01A97D
:103460002046FFF7C2FE074607B130E02046FFF7CF
:1034700017FE0746A069C67A97B1042F00D026E050
:1034800006F0200038B10020A0606061002706F03F
:10349000040020B9E3E706F0040000B9052716E0B0
:1034A00006F0040000B112E06569E87A00F010004F
:1034B00008B905270BE0A97EE87E41EA00212A7DB4
:1034C000687D42EA002041EA0040A060C7E700BFF3
:1034D0003846BDE8FC8170B504460D46607801238E
:1034E0002A4604F1340101F068FF08B1032070BDE1
:1034F00094F8321294F8330241EA00204AF655213A
:10350000884201D00220F2E794F86D00010694F899
:103510006C0041EA004194F86B0041EA002094F805
:103520006A10084320F07F407649884201D100208C
:10353000DDE794F88900010694F8880041EA00412B
:1035400094F8870041EA002094F88610084320F0A0
:103550007F406C49884201D10020C8E70120C6E7BE
:103560002DE9F74F88B0089800680190019800781D
:1035700030380790079809280AD8019840783A28E7
:1035800006D10198801C019008990198086002E01A
:103590005D4800780790079818B10B200BB0BDE884
:1035A000F08F5A49079851F82040099804600CB9E7
:1035B0000C20F3E7207878B1607801F0FBFE8046BC
:1035C00008F0010040B90A9820B108F0040008B1E1
:1035D0000A20E3E70020E1E70020207007986070F0
:1035E000607801F0CBFE804608F0010008B10320AE
:1035F000D4E70A9820B108F0040008B10A20CDE70A
:103600004FF0000B59462046FFF765FF054600BF07
:10361000012D21D14FF0000ABAF1000F03D0AAF119
:10362000010000F0FF0A4FF4DF7000EB0A1104F113
:1036300034000F18387978B1F87A0106B87A41EA7F
:103640000041787A41EA0020397A40EA010B594674
:103650002046FFF740FF0546032D01D101209DE7DD
:103660000DB10D209AE73F20015D94F8400041EA3A
:103670000020B0F5007F01D00D208FE74A20015DCA
:1036800094F84B0041EA0029B9F1000F0ED194F8EB
:103690005B00010694F85A0041EA004194F8590091
:1036A00041EA002094F8581040EA0109C4F820903B
:1036B0004420065DE670012E03D0022E01D00D20BD
:1036C0006CE709FB06F94120005D0646A07016B1C3
:1036D000701E304008B10D2060E74520015D94F870
:1036E000460041EA00202081207A00F00F0078B1E6
:1036F0000D2053E7222A2B2C3A3B3C3D3E3F5B5D9D
:103700007C7F0000464154004E000020480000200D
:103710004720015D94F8480041EA00200690069891
:1037200070B994F85700010694F8560041EA004138
:1037300094F8550041EA002094F85410084306908C
:103740004220015D94F8430041EA00200290029873
:1037500008B90D2022E702984844218900EB111096
:103760000590DDE90501814201D20D2016E7DDE972
:103770000510401AA178B0FBF1F00490049808B944
:103780000D200BE7012540F6F6710498884200D31E
:1037900002254FF6F6710498884200D30325049859
:1037A000801CE06105985844E062029858446062C9
:1037B000032D16D1208908B10D20EFE694F863009F
:1037C000010694F8620041EA004194F8610041EA80
:1037D000002094F860100843A062E0698000039024
:1037E00014E0208908B90D20D8E6606A4844A06238
:1037F000022D02D1E069400007E0207F00F00100C7
:10380000E16901EB410100EB51000390216A03984B
:1038100000F2FF10B1EB502F01D20D20BEE64FF0A9
:10382000FF3020610020E060032D5CD1607194F8CE
:10383000641094F8650041EA0020584460616078A3
:10384000012304F13401626901F0B7FDF0BB94F883
:10385000321294F8330241EA00204AF65521884298
:1038600041D13720005D01063620005D41EA00416C
:103870003520005D41EA002094F834100843FE49E9
:10388000884230D194F81B02010694F81A0241EAEA
:10389000004194F8190241EA002094F818120843F4
:1038A000F64988421FD194F82302010694F82202B7
:1038B00041EA004194F8210241EA002094F82012E4
:1038C0000843E06094F81F02010600E00BE094F862
:1038D0001E0241EA004194F81D0241EA002094F8DA
:1038E0001C12084320612570E5480088401C80B206
:1038F000E3490880E080002020632071A06100BFC0
:103900004CE670B504460D4624B1207810B1E0882D
:10391000A84201D0092070BD607801F04BFD00F095
:10392000010008B10320F6E70020F4E70246012A6F
:1039300001DB0B207047D34850F822300BB1002038
:10394000187009B100200870CE4840F822100020FD
:10395000F0E72DE9F7438AB00546164600202860B7
:1039600006F01F0626F0010203A90BA8FFF7F8FDD9
:103970000746CDF824D027B903A80B99FFF74EFDD1
:103980000746089C0FB904B9062706F01C0000285A
:1039900058D04FB1042F03D103A8FFF7D9FB074636
:1039A00046F00806089C09E0E07A00F0110008B132
:1039B000072703E006F0040000B10827002F40D1DC
:1039C00006F0080000283CD001F0AAFD804684F8EB
:1039D0000E804FEA1821E1734FEA184121744FEA33
:1039E000186161740020E072207700216177A1776F
:1039F000E177A17EE07E41EA0021227D607D42EAFE
:103A0000002041EA00490020A0760021E1762075DF
:103A10006175012003990871B9F1000F11D0039865
:103A2000D0F8308049460398FFF7AEF9074647B90A
:103A3000A9F101000399C86041460398FEF7ECFF25
:103A400007460EE06FB9E07A00F0100008B10427D5
:103A500007E006F0020020B1E07A00F0010000B1BA
:103A6000072747B906F0080008B146F0200603987A
:103A7000006BE8612C62FFB9AE71A17EE07E41EA85
:103A80000021227D607D42EA002041EA0040286159
:103A9000E07F0106A07F41EA0041607F41EA00200B
:103AA000217F0843E8600020A860A861686203984D
:103AB00028600398C088A88038460DB0BDE8F08320
:103AC0002DE9FF4F83B0044615469A46DDF810B045
:103AD0000020CAF80000A1882068FFF712FF0290BA
:103AE000029818B1029807B0BDE8F08FA07900F0F5
:103AF000800008B10220F6E7A07900F0010008B9C3
:103B00000720F0E7D4E90210401A0090009885429F
:103B100000D9009DC6E02089C0F30800002870D1BC
:103B200020688078401EA16800EA512000F0FF095B
:103B3000B9F1000F25D1A06810B9206901900CE0FF
:103B4000606A28B12046A168FFF7B7F9019004E048
:103B500061692068FFF70BF801900198022805D2EF
:103B6000A07940F08000A0710220BCE70198401CC1
:103B700028B9A07940F08000A0710120B3E7019836
:103B8000606161692068FEF7E5FF06462EB9A079FD
:103B900040F08000A0710220A5E74E444FEA55286E
:103BA000B8F1000F2ED009EB08002168897888420F
:103BB00003D920688078A0EB090808F0FF0321688A
:103BC00048783246594601F0F8FB28B1A07940F018
:103BD0008000A071012086E7A07900F0400068B164
:103BE000A069801B404509D2A169891B0BEB4120CC
:103BF0004FF4007204F12801FEF7DAFE4FEA48277D
:103C000046E029E0A069B04225D0A07900F040004C
:103C100090B121684878012304F12801A26901F0DC
:103C200003FC28B1A07940F08000A07101205AE780
:103C3000A07920F04000A071216848780123324625
:103C400004F1280101F0B9FB28B1A07940F080000F
:103C5000A071012047E7A6612089C0F30800C0F5E4
:103C60000077AF4200D92F462089C0F3080204F143
:103C7000280011183A4607E05252614172724161C0
:103C80004C000020480000205846FEF791FE00BF7F
:103C9000BB44A0683844A060DAF800003844CAF891
:103CA0000000ED1B002D7FF436AF00201BE72DE94F
:103CB000FF4F83B0044615469B46049801900020B0
:103CC000CBF80000A1882068FFF71BFE0290029845
:103CD00018B1029807B0BDE8F08FA07900F080001D
:103CE00008B10220F6E7A07900F0020008B9072029
:103CF000F0E7E0682844E168884200D20025D6E079
:103D00002089C0F3080000287ED120688078401EFA
:103D1000A16800EA512000F0FF0ABAF1000F32D189
:103D2000A06858B9D4F81080B8F1000F13D1002161
:103D30002068FFF75DF8804620610CE0606A28B1DA
:103D40002046A168FFF7B9F8804604E06169206861
:103D5000FFF74EF88046B8F1000F00D1AAE0B8F1A5
:103D6000010F05D1A07940F08000A0710220B1E7D9
:103D700008F1010028B9A07940F08000A07101206D
:103D8000A8E7C4F81480A07900F0400090B1216841
:103D90004878012304F12801A26901F045FB28B10C
:103DA000A07940F08000A071012093E7A07920F075
:103DB0004000A07161692068FEF7CCFE06462EB96E
:103DC000A07940F08000A071022083E756444FEABA
:103DD0005529B9F1000F30D00AEB09002168897824
:103DE000884203D920688078A0EB0A0909F0FF0314
:103DF000216848783246019901F016FB38B1A07964
:103E000040F08000A07100E02EE0012062E7A06990
:103E1000801B48450ED2A069801B019A02EB40210D
:103E20004FF4007204F12800FEF7C2FDA07920F0E3
:103E30004000A0714FEA49272DE0A069B04212D09E
:103E4000D4E9020188420ED2216848780123324623
:103E500004F1280101F0B1FA28B1A07940F0800006
:103E6000A071012036E7A6612089C0F30800C0F5E3
:103E70000077AF4200D92F462189C1F3080204F12F
:103E8000280150183A460199FEF792FDA07940F0BA
:103E90004000A07100BF019838440190A0683844E8
:103EA000A060DBF800003844CBF80000ED1B002DCB
:103EB0007FF426AF00BFD4E90201884201D9A0688F
:103EC000E060A07940F02000A071002002E72DE919
:103ED000F0410446A1882068FFF713FD0746002F34
:103EE0004FD1A07900F0200000284AD0A07900F03E
:103EF000400078B121684878012304F12801A269C3
:103F000001F092FA10B10120BDE8F081A07920F013
:103F10004000A071E1692068FEF77EFD0746002F92
:103F20002FD1256AE87A40F02000E872207B2877BC
:103F3000A089010A6977E068010CA977E068010EA1
:103F4000E977207CA876208A010AE9762069000CAE
:103F500028752069010E697501F0E2FA0646AE7512
:103F6000310AE975310C2976310E6976A07920F095
:103F70002000A0710120216808712068FEF785FDEE
:103F800007463846C0E770B504462046FFF79FFF56
:103F900005460DB900202060284670BD0146012964
:103FA00001DB0B207047FE4801700020FAE711B5D5
:103FB0008BB0002204A90BA8FFF7D2FA04462CBB51
:103FC00001A80A9004A80B99FFF728FA0446D4B96F
:103FD000099818B904990698886114E00998C07A7C
:103FE00000F0100070B10998817EC07E41EA002186
:103FF0000998027D407D42EA002041EA0040049990
:10400000886100E00524042C00D1052420460CB072
:1040100010BD2DE9FE4F04460D46A1882068FFF72C
:1040200070FC0290029810B10298BDE8FE8FA07952
:1040300000F0800008B10220F7E7606A00287DD018
:10404000681C002841D1D4F8248058F804AB4FF004
:10405000020926696EB300BF00964FF0000B09F10C
:10406000020900BF01960BF1010B31462068FEF7F3
:104070007EFD0646012E05D8A07940F08000A07193
:104080000220D2E7701C28B9A07940F08000A0710E
:104090000120CAE70198401C8642E3D0D14504D8EC
:1040A00048F804BB009848F8040B2068C069B04287
:1040B000D2D8606AC0F80090D14503D80020C8F873
:1040C000000050E0112002904DE0E068A84200D2CC
:1040D000E568A560002D46D0691E2046FEF7EDFE7E
:1040E000606161692068FEF735FD07462FB9A07948
:1040F00040F08000A071022097E720688078401E81
:10410000691E00EA512007442089C0F3080050B31B
:10411000A069B84227D0A07900F0400098B121688A
:104120004878012304F12801A26901F07DF930B13A
:10413000A07940F08000A071012076E714E0A0791A
:1041400020F04000A0712168487801233A4604F12C
:10415000280101F032F928B1A07940F08000A07167
:10416000012062E7A761C1E0E068A84204D2A0791B
:1041700000F0020000B9E568D4F808904FF000089C
:10418000C4F80880002D77D0206880784702B9F104
:10419000000F11D0681EB0FBF7F1A9F10100B0FBD0
:1041A000F7F0814208D3A9F10100791E8843A0608D
:1041B000A0682D1A666918E02669AEB9002120684A
:1041C000FEF716FE0646012E05D1A07940F08000CC
:1041D000A071022029E7701C28B9A07940F0800066
:1041E000A071012021E726616661EEB329E0A07984
:1041F00000F0020038B131462068FEF7F9FD0646AE
:1042000036B93D461FE031462068FEF7B0FC064651
:10421000701C28B9A07940F08000A071012004E74B
:10422000012E03D92068C069B04205D8A07940F0BA
:104230008000A0710220F8E66661A0683844A060A2
:10424000ED1BBD42D3D800BFA0682844A060C5F3D1
:10425000080048B131462068FEF77CFC8046B8F182
:10426000000F07D1A07900E006E040F08000A071C7
:104270000220DAE608EB55282089C0F3080050B385
:10428000A069404527D0A07900F0400090B1216896
:104290004878012304F12801A26901F0C5F828B18A
:1042A000A07940F08000A0710120BEE6A07920F046
:1042B0004000A071216848780123424604F128019A
:1042C00001F07BF828B1A07940F08000A0710120B6
:1042D000ABE6C4F81880D4E90201884205D9A06889
:1042E000E060A07940F02000A07100BF02989CE639
:1042F00033B583B004460022214604A8FFF730F905
:1043000005464DBBC4F818D020460499FFF786F83F
:104310000546F5B9606998B16069C07A00F010008F
:1043200068B16069817EC07E41EA00216069027DDA
:10433000407D42EA002041EA0040A06000E00525FF
:104340003DB92068C088A08000212046FEF7CEFD40
:104350000546042D00D10525284605B030BDFEB523
:1043600004460E46A1882068FFF7CBFA05461DBB20
:104370002EB900212046FEF7B9FD05461CE0C4F821
:1043800018D02046FEF7BAFE0546042D02D10020C3
:104390002061002585B931462046FEF7F3FF01E094
:1043A0004E00002000212046FEF7EEFD0546042DBC
:1043B00002D10020206100252846FEBD33B58BB018
:1043C0000D46002204A90BA8FFF7CAF804467CB9E1
:1043D00001A80A9004A80B99FFF720F804463CB9FD
:1043E000099820B1294604A8FEF7CCFF00E0062476
:1043F00020460DB030BD2DE9F74F82B08B461446F4
:104400000022214602A8FFF7ABF80190019800288E
:1044100077D120680169C069801E814204D8206874
:104420000069CBF800006CE0206890F800A000263E
:10443000BAF1010F1DD1022700BF39462068FEF7EF
:1044400096FB804608F1010010B9012001900FE0B1
:10445000B8F1010F02D10220019009E0B8F1000F7C
:1044600000D1761C781C07462168C9698842E4D3CC
:104470003DE02068C7692068406A00904FF000095D
:10448000002500BFB9F1000F0FD1009A531C11464F
:1044900000932068FEF7C0FA0190019800B125E072
:1044A000206800F134054FF40079BAF1020F09D108
:1044B0002878697840EA012000B9761CAD1CA9F182
:1044C000020910E0E8780006A97840EA014069781E
:1044D00040EA01202978084320F0704000B9761C9A
:1044E0002D1DA9F10409781E071ECBD100BF20683D
:1044F0000661BAF1030F02D1012021684871CBF89F
:104500000060019805B0BDE8F08F70B50446A18841
:104510002068FFF7F6F9054655B9A07900F080004C
:1045200008B1022504E0A07900F0020000B90725D7
:10453000002D36D1D4E9021088422DD9A068E06060
:10454000A07940F02000A071A06838B921692068E6
:10455000FEF71AFC0546002020611DE06169206815
:10456000FEF705FB06460025701C00B90125012E4B
:1045700000D1022585B92068C069B0420CD96FF01E
:10458000704261692068FEF764FB054625B9314633
:104590002068FEF7F9FB05461DB1A07940F08000C8
:1045A000A071284670BD71B591B001220AA911A869
:1045B000FEF7D6FF0446002C55D1CDF840D00AA80E
:1045C0001199FEF72BFF04462CB91098C07A00F021
:1045D000200000B10624002C45D10F9D0DB9062402
:1045E00004E0E87A00F0010000B10724A97EE87E2B
:1045F00041EA00212A7D687D42EA002041EA004626
:1046000004BBE87A00F01000E0B1022E01D20224CF
:1046100018E01C220AA903A8FEF7CAF90596022190
:1046200003A8FEF763FC044664B903A8FEF766FD21
:1046300004461CB103988069B04200D10724042CC1
:1046400000D100247CB90AA8FEF7B9FD044654B98C
:1046500026B131460A98FEF797FB04461CB90A9822
:10466000FEF713FA0446204612B070BD2DE9F1475B
:104670008BB000F055FF0746012204A90BA8FEF7F6
:104680006FFF0646002E73D101A80A9004A80B996B
:10469000FEF7C4FE064606B90826042E05D10A9880
:1046A000C07A00F0200000B10626042EEBD10021D4
:1046B0000498FEF79DFB0546002605B90726012D47
:1046C00000D10226681C00B9012626B900210498F1
:1046D000FEF7A2F90646002E68D129460498FEF797
:1046E00039FA8246049800F134044FF40072002134
:1046F0002046FEF76AF90B2220212046FEF765F9D5
:104700002E2020701020E072A775390AE175390C4F
:104710002176390E6176A576290AE176280C207576
:10472000290E61752022214604F12000FEF740F990
:104730002E2084F82100DDF81880049800780328E2
:1047400004D10498806A404500D1B04684F83A808C
:104750004FEA182184F83B10C8F307413420015573
:104760004FEA186184F83510049890F8029019E027
:104770003FE00498C0F830A00AF1010A0120049932
:10478000087100210498FEF747F9064606B10CE0CF
:104790004FF4007200212046FEF717F9A9F101003D
:1047A00000F0FF09B9F1000FE3D100BF1EB904A862
:1047B000FEF7CEFC064626B129460498FEF7E4FA39
:1047C00017E0099C1020E072A775390AE175390CD1
:1047D0002176390E6176A576290AE176280C2075B6
:1047E000290E61750120049908710498FEF74DF9AE
:1047F000064630460CB0BDE8F087F7B58AB00F46E4
:104800001446012203A90AA8FEF7AAFE05460DBB1D
:10481000CDF824D003A80A99FEF700FE05462DB96D
:104820000998C07A00F0200000B1062595B9089ECD
:104830000EB906250EE004F0270407EA0400F17A19
:10484000A1430843F0720120039908710398FEF711
:104850001CF9054628460DB0F0BD73B58AB00D466B
:10486000012203A90AA8FEF77BFE06461EBBCDF86F
:1048700024D003A80A99FEF7D1FD06462EB909985F
:10488000C07A00F0200000B10626A6B9089C0CB939
:10489000062610E0A879A075E8880112E17528794C
:1048A0002076A88801126176012003990871039887
:1048B000FEF7EBF8064630460CB070BDF3B597B086
:1048C0000F46012210A917A8FEF74AFE0546002D43
:1048D00014D110980990CDF858D010A81799FEF768
:1048E0009DFD05462DB91698C07A00F0200000B154
:1048F0000625002D76D1159808B9042572E0159883
:1049000000F10B01152203A8FEF752F81C2210A992
:1049100009A8FEF74DF8394609A8FEF77FFD0546C0
:1049200005B90825042D5DD109A8FEF711FC05463F
:10493000002D57D10E9C13220DF10E0104F10D0034
:10494000FEF736F89DF80C0040F02000E0720120E0
:10495000109908710B991298884239D0E07A00F0CA
:104960001000002834D0A37EE27E43EA022394F8AC
:1049700014C0627D4CEA022243EA02410998FEF724
:10498000E9F806460EB9022522E031460998FEF7FD
:1049900043F80546099800F15404CDB960782E28F3
:1049A00016D109980078032806D109990B98896ACD
:1049B000884201D1002000E00B980646A676310A15
:1049C000E176300C2075310E61750120099908716E
:1049D00045B910A8FEF7F3FB05461DB91098FEF780
:1049E00054F80546284619B0F0BD2DE9F74F8EB0B2
:1049F00091460E98012803DB0B2011B0BDE8F08F23
:104A00000F98012801DD1320F7E7A9F1010000EA62
:104A1000090008B11320F0E7FE490E9851F820B0C4
:104A2000BBF1000F01D10C20E7E700208BF800005C
:104A30000E980B9000200A900B9800F09FFC0090BD
:104A4000009800F0010008B10320D6E7009800F0BC
:104A5000040008B10A20D0E700BF03AA01210B9887
:104A600000F00FFD10B90398802801D20120C4E79F
:104A70000F9808B1002000E03F2080460398A0EB8B
:104A800008000390B9F1000F13D14FF4FA610398B5
:104A9000B0FBF1F009904FF0000A01E00AF1010AC1
:104AA000DD4830F81A1009988142F7D8DB4830F811
:104AB0001A904FEA5929B9F1000F01D14FF00109BD
:104AC000B9F1800F01D94FF080090398B0FBF9F7D5
:104AD000012540F6F670874200D302254FF6F670A6
:104AE000874200D30325032D0AD1082000EB87005D
:104AF00000F2FF10460A202002900020019011E0F1
:104B0000012D05D107EB4700401C4008C01C01E007
:104B10007800001D064606F2FF10460A01200290AA
:104B20002020019002984044069006983044059059
:104B3000019905980844049004984844A0EB0800A3
:104B40000399884201D90E2057E708AA03210B9840
:104B500000F097FC28B9089818B10898B0F5004FF4
:104B600001D901200890089904980844401E491E64
:104B70008843089008990498081A0890032D08D1D2
:104B800008990298084402900899069808440690EB
:104B900001E008980644DDE90201081A811B01982A
:104BA000081AB0FBF9F7022D03D140F6F6708742E0
:104BB00005D3032D05D14FF6F670874201D20E20A2
:104BC0001BE7012D02D0022D0CD102E001200C9038
:104BD0000BE00398B0F5803F01D2042000E00620EE
:104BE0000C9002E00C200C9000BF00BF00BF0F989B
:104BF00010B1F0200D9044E04FF4007200210BF151
:104C00003400FDF7E2FE0BF5F97401206070A0702E
:104C10000020E0700C982071FE20607103984044E1
:104C20003F21B0FBF1F0FF21B0FBF1F008903F21F4
:104C3000089841EA9000A0710898E0713F20207226
:104C400000216172A172E172039820730398010A36
:104C500061730398010CA1730398010EE173552150
:104C60008BF83212AA218BF83312012300220BF1A8
:104C700034010B9800F0D8FB08B10120BDE6F82004
:104C80000D900BF134044FF4007200212046FDF723
:104C90009CFE0B2262A12046FDF78AFE4FF4007AAB
:104CA00084F80BA04FEA1A21217384F80D90029822
:104CB000A0730298010AE17301202074032D01D131
:104CC000002001E04FF40070824684F811A04FEA02
:104CD0001A21A1740398B0F5803F05D20398E074BF
:104CE0000398010A217510E0039884F820000398C6
:104CF000C0F30721212001550398C0F3074122206A
:104D000001550398010E232001550D9860753F2031
:104D1000207600216176FF20A076E17684F81C8061
:104D20004FEA182161774FEA1841A1774FEA1861DD
:104D3000E17700F0F5FB0890032D3ED1089884F848
:104D400043000898C0F30721442001550898C0F398
:104D50000741452001550898010E4620015584F869
:104D60002460C6F3072125200155C6F307412620FC
:104D70000155310E27200155022084F82C00002116
:104D80002D2001552E2001552F200155012084F89A
:104D9000300031200155062084F8320033200155BF
:104DA000802084F84000292084F8420013221FA1AB
:104DB00004F14700FDF7FCFD1FE0089884F8270088
:104DC0000898C0F30721282001550898C0F307412F
:104DD000292001550898010E2A200155A675310A8F
:104DE000E175802084F82400292084F8260013220D
:104DF00013A104F12B00FDF7DBFD552084F8FE0123
:104E0000AA2140F2FF1001550123424621460B988A
:104E100020E0000048000020F46300080A64000855
:104E2000EBFE904D53444F53352E30004E4F204EE5
:104E3000414D45202020204641543332202020007F
:104E40004E4F204E414D45202020204641542020E9
:104E50002020200000F0E8FA08B10120CDE5032D64
:104E600006D1012308F1060221460B9800F0DCFA76
:104E7000069807904FF0000A61E04FF4007200219D
:104E80002046FDF7A2FD0D980890032D14D0012DAA
:104E900001D1FE4801E06FF0FF0008990843089037
:104EA000089820700898000A60700898000CA0709C
:104EB0000898000EE07019E0089860F0FF00089074
:104EC000089820700898000A60700898000CA0707C
:104ED0000898000EE070FF202071FF216171A17120
:104EE000E17120726172A1720F21E1720798411C79
:104EF00002460123079121460B9800F095FA08B16C
:104F000001207AE54FF4007200212046FDF75DFD97
:104F1000012008900EE00798411C024601230791EA
:104F200021460B9800F080FA08B1012065E5089849
:104F3000401C08900898B042EDD30AF1010ABAF17A
:104F4000000F9AD0032D01D1484600E00198824617
:104F500000BF0798411C02460123079121460B9888
:104F600000F062FA08B1012047E5AAF10100B0F1B2
:104F7000000AEED1032D46D15220207060706120CE
:104F8000A0704120E070722084F8E401722140F2A8
:104F9000E51001554121401C01556121401C01557E
:104FA000781E84F8E801C0F3072140F2E9100155AA
:104FB000781EC0F307414FF4F5700155781E010EBD
:104FC00040F2EB100155022084F8EC01002140F280
:104FD000ED100155401C0155401C0155552084F829
:104FE000FE01AA2140F2FF100155012308F1010240
:104FF00021460B9800F018FA012308F10702214618
:105000000B9800F011FA002211460B9800F039FAC3
:1050100008B10120F1E40020EFE42DE9FC47074648
:105020008846914600243E4611E06B46012201A9C4
:105030004846FEF745FD0098012800D00BE09DF89A
:10504000045006F8015B641C0A2D00D103E0A8F1AE
:105050000100A042E9DC00BF0020307014B13846E6
:10506000BDE8FC870020FBE77CB504460D468DF8C3
:105070000040012601AB324669462846FEF717FE7E
:105080000198B04200D17CBD4FF0FF30FBE770B516
:1050900004460E4600250AE020783146FFF7E4FF7B
:1050A000401C10B94FF0FF3070BD641C6D1C20789F
:1050B0000028F1D12846F7E70FB42DE9F04F89B069
:1050C00014A8089000208146019044E1139810F83C
:1050D000014B139004B943E1252C0AD020461299C4
:1050E000FFF7C2FF814609F1010008B14FF0010945
:1050F0002EE1002006468246139810F8014B1390CB
:10510000302C05D10126139810F8014B139006E0BE
:105110002D2C04D10226139810F8014B139009E0AE
:105120000AEB8A0004EB4000A0F1300A139810F853
:10513000014B1390302C01DB392CF1DD6C2C01D0AC
:105140004C2C05D146F00406139810F8014B13902F
:1051500004B905E12546612D04DB7A2D02DCA5F1B9
:105160002000C5B24F2D59D006DC422D53D0432D1F
:1051700047D0442D5CD154E0532D04D0552D51D04F
:10518000582D55D151E00898006802900898001DEC
:1051900008904FF0000801E008F10108029810F8AB
:1051A00008000028F8D1009006F0020068B907E076
:1051B00020201299FFF758FF81460099084400907B
:1051C000404608F101085045F2D312990298FFF7C2
:1051D0005EFF814600990844009007E02020129964
:1051E000FFF742FF8146009908440090404608F1CD
:1051F00001085045F2D309F1010008B1DDF8009033
:10520000A6E0089911F8042BD0B208911299FFF783
:105210002BFF81469CE0022007900FE008200790BA
:105220000CE000BF0A20079008E01020079005E07E
:1052300020461299FFF718FF814689E000BF06F06B
:10524000040028B1089800680899091D08910CE02D
:10525000442D05D1089800680899091D089104E0BB
:10526000089800680899091D08918346442D06D1C5
:105270000BF0004018B1CBF1000B46F008060027F8
:1052800000BF0798BBFBF0F102E0000000FFFF0049
:1052900000FB11B0C5B20798BBFBF0FB092D06DD82
:1052A000782C01D1272000E007202844C5B205F161
:1052B0003000C2B238467F1C03A90A54BBF1000F6C
:1052C00001D0102FDDD306F0080020B12D22384682
:1052D0007F1C03A90A54B84606F0010008B130202B
:1052E00000E0202005460020019007E028461299A2
:1052F000FFF7BAFE814601990844019006F00200CA
:1053000020B9404608F101085045EFD300BF791E8F
:105310000F4603AA505C1299FFF7A6FE8146019939
:1053200008440190002FF2D107E020201299FFF7E6
:105330009BFE8146019908440190404608F101080E
:105340005045F2D309F1010008B1DDF8049000BF27
:1053500001984844019009F1010000287FF4B6AE9D
:1053600000BF0020089009F1010028B9484609B0A3
:10537000BDE8F00F5DF814FB0198F8E770B504463E
:10538000002514B1012C0DD10BE0FCF705FE0546FC
:1053900035B1FCF7CFFCFF20FCF7C6FCFCF7CFFCD7
:1053A00002E001E0012500BF00BF0DB1012070BD8A
:1053B0000020FCE70146002070472DE9F041074638
:1053C0000D4616461C464FF0000814B90420BDE8EF
:1053D000F08117B1012F1CD110E02246314628463A
:1053E000FCF79BFE8046B8F1000F06D0FCF7A2FC4C
:1053F000FF20FCF799FCFCF7A2FC0DE004E0761C12
:1054000005F50075601EC4B2002CF8DC4FF00008F2
:1054100002E04FF0010800BF00BFB8F1000F01D15A
:105420000020D4E70120D2E72DE9F04107460D46E0
:1054300016461C464FF0000814B90420BDE8F08160
:1054400017B1012F12D106E0224631462846FCF75B
:10545000A0FE80460DE004E0761C05F50075601E98
:10546000C4B2002CF8DC4FF0000802E04FF0010855
:1054700000BF00BFB8F1000F01D10020DEE701201E
:10548000DCE72DE9F04106460F4615463EBB37B135
:10549000012F1CD0022F11D0032F1DD113E040216A
:1054A0002048FBF711FBFCF75FFC08B9002400E083
:1054B000012440211B48FBF705FB0FE04FF400706F
:1054C000288000240AE008202880002406E0FCF759
:1054D00028FD2860002401E0042400BF1DE0012E07
:1054E0001AD137B1012F0FD0022F04D0032F10D1C2
:1054F00006E000240FE04FF40070288000240AE04A
:1055000008202880002406E007480088286000243E
:1055100001E0042400BF00E001242046BDE8F08142
:1055200000207047000802405000002010B50446DB
:105530000848406800F07F40B0F1006F08D1606813
:10554000054908602068FAF7FEFD034800688047B7
:1055500010BD00000000010854000020D2B201E09C
:1055600000F8012B491EFBD270470022F6E710B568
:1055700013460A4604461946FFF7F0FF204610BDC1
:10558000421C10F8011B0029FBD1801A704730B56E
:105590000B46014600202022012409E021FA02F5F1
:1055A0009D4205D303FA02F5491B04FA02F528448B
:1055B000151EA2F10102F1DC30BD2DE9F05F0546B8
:1055C000002092469B4688460646814640241BE0C2
:1055D000284641464746224600F0F9F953465A46C6
:1055E000C01A914110D311461846224600F0E0F946
:1055F0002D1A67EB01084F4622460120002100F0DA
:10560000D7F917EB00094E41201EA4F10104DFDC9D
:10561000484631462A464346BDE8F09F2DE9FE4FF5
:10562000804681EA0300C00F0C46009021F0004143
:1056300023F00045B8EB0200A94105D240462146BF
:1056400090461C460B46024623F00040104347D0CC
:10565000270DC7F30A00C3F30A510290401A0190C4
:1056600040286BDAC3F3130040F4801B0098924685
:1056700020B10023D2EB030A63EB0B0B01985946D0
:10568000C0F14002504600F093F906460D465046E0
:105690005946019A00F0ABF910EB08006141002473
:1056A00087EA115284EAE7731A4340D0009A62B342
:1056B000019A012A4FEA075215DC001B61EB020137
:1056C0004FF0004202EA0752CDE90042001C41F5CA
:1056D000801132462B4600F0ABF903B0BDE8F08FE5
:1056E00040462146F9E7001B61EB0201001C41F531
:1056F000801300185B412018A2F5001747EB030147
:1057000040EAD570B6196D4111E06D084FEA3606D2
:1057100045EAC0754FEA0752001B61EB0201001C0D
:1057200041F5801149084FEA3000001951413246D5
:105730002B4603B0BDE8F04F00F06BB90098012292
:1057400040000023D0EB020263EBE0730098214697
:105750004FEAE074B8EB000061EB0401E9E783F085
:1057600000435BE781F0004158E72DE9FE4F81EAF5
:10577000030404F0004421F0004100944FF0000BBA
:1057800023F0004350EA01045ED052EA03045BD0E8
:10579000C3F30A54C1F30A552C44A4F2F334019420
:1057A000A0FB0254C1F3130141F48011C3F31303AE
:1057B00043F4801301FB024400FB034E840A970A62
:1057C00044EA815447EA8357A4FB076802958D0A8F
:1057D00005FB07854FEA932C04FB0C542705029D1B
:1057E0004FEA065847EA1637B5EB08056EEB070C8B
:1057F000870E920E47EA811742EA8312A7FB020145
:10580000B6EB0B0164EB00042B0D43EA0C335E187E
:1058100044EB1C50DA465146E7FB0201C5F3130482
:105820004FEA0B3343EA14534FEA0432019C43EA34
:105830000603A4F10C040294009CCDE900B400F02E
:10584000F7F803B0BDE8F08F00200146F9E72DE935
:10585000F04D81EA030404F0004B21F000451446AA
:105860004FF0000A23F0004150EA050220D054EA2C
:1058700001021DD0C5F30A570246C5F31303C1F355
:105880001300C1F30A5640F4801543F48013A7EBCC
:105890000608101BD64608F2FD3873EB050002D34C
:1058A00008F1010801E092185B41B8F1000F03DA3A
:1058B00000200146BDE8F08D00204FF4801106461F
:1058C00084460EE0171B73EB050705D3121B63EB31
:1058D000050306434CEA010C49084FEA30009218D0
:1058E0005B4150EA0107EDD152EA030012D082EA8F
:1058F000040083EA0501084305D0101BAB4106D222
:105900000122002306E000224FF0004302E06FF086
:10591000010253101AEB06004CEB085110EB0A0081
:1059200041EB0B01BDE8F04D00F073B8C1F30A5232
:10593000C1F3130140F2FF3341F480119A4202DABD
:1059400000200146704740F233439A42A2F23342AC
:1059500002DC524200F03BB800F02AB830B5041E19
:1059600071F1000404DB4FF00044404264EB01019C
:10597000141E73F1000405DB1C464FF00043524235
:1059800063EB0403994208BF904230BD064C074DBB
:1059900006E0E06840F0010394E8070098471034FF
:1059A000AC42F6D3FAF7C2FB20640008406400085A
:1059B000202A04DB203A00FA02F1002070479140CF
:1059C000C2F1200320FA03F3194390407047202AC4
:1059D00004DB203A21FA02F00021704721FA02F399
:1059E000D040C2F120029140084319467047202A56
:1059F00006DBCB17203A41FA02F043EAE07306E0F7
:105A000041FA02F3D040C2F1200291400843194606
:105A1000704710B5141E73F1000408DA401C41F100
:105A2000000192185B411A4301D120F0010010BD22
:105A30002DE9F04D92469B4611B1B1FA81F202E098
:105A4000B0FA80F220329046FFF7B2FF04460F46CC
:105A500040EA0A0041EA0B0153465A46084313D074
:105A6000114653EA010019D0C8F140025046FFF731
:105A7000AEFF05460E46504659464246FFF798FF90
:105A8000084305D0012004E020463946BDE8F08DEA
:105A90000020054346EAE0762C4337430A98630525
:105AA000E40AA0EB08000022FD0A44EA47540A3049
:105AB00002D500200146E9E7010510196941DDE939
:105AC000084500196941BDE8F04DA2E70FB4084B45
:105AD00010B504A902AA039800F0F0F8044602A940
:105AE000002000F082FC204610BC5DF814FB000092
:105AF000EB63000837B514460846064B6A46214654
:105B000000F0DCF804466946002000F06EFC2046F8
:105B10003EBD0000EB63000802E008C8121F08C188
:105B2000002AFAD170477047002001E001C1121F1E
:105B3000002AFBD1704700002DE9FF5F82B00021F1
:105B4000DDE90430020DDDF840B0034318D044F61F
:105B50001050A2F2FF3242431514119801281FD0B1
:105B6000A5EB0B00401C5FEA000A4FF000064E4F09
:105B7000DFF83891B046504615D5CAF1000413E05D
:105B8000119801244AA3012801D16FEA0B01029860
:105B9000119AC0E90031C0E9024206B0BDE8F09FA9
:105BA000CBF10000DFE704460021404A491842EBF0
:105BB0000450CDE9001012E0E00707D032463B4622
:105BC00040464946FFF7D1FD8046894632463B466E
:105BD00010461946FFF7C9FD06460F466410002C13
:105BE000EAD1DDE90401DDE90023BAF1000F06DAAC
:105BF000FFF7BBFD42464B46FFF7B7FD05E0FFF759
:105C000026FE42464B46FFF722FE04460E46002281
:105C1000284BFFF7A3FE03D84FF0FF30014607E003
:105C20000022254B20463146FFF7F8FCFFF77EFEA9
:105C3000102409E0002C0ADB0A220023FFF7BDFC38
:105C4000039B30321A55641E50EA0102F2D1641CE3
:105C5000039AC4F111031444119A012A03D00122BA
:105C600008430DD10AE0084304D000204FF0110B87
:105C7000119072E7A3EB0B056D1E0DE05B4504DD93
:105C80004FF0000205F1010504E003DA4FF00002D5
:105C9000A5F10105002AECD002981199C0E9023162
:105CA000C0E9004579E70000000014400000F03F23
:105CB000300000000000F0430000E03F2DE9FF4FFE
:105CC00095B09B468946064600250FE2252877D1E8
:105CD00000242746F84A0121059400E0044316F801
:105CE000013F203B01FA03F01042F7D130782A2817
:105CF00011D06FF02F033078A0F13002092A16D8A6
:105D0000059A44F0020402EB820203EB42021044C3
:105D1000761C0590EFE759F8042B0592002A03DA68
:105D2000504244F40054059044F00204761C30784C
:105D30002E2816D116F8010F44F004042A280DD09D
:105D40006FF02F023078A0F13003092B09D807EB50
:105D5000870302EB4303C718761CF3E759F8047B6B
:105D6000761C30786C280FD006DC4C2817D06828B9
:105D70000DD06A2814D104E0742810D07A280FD1ED
:105D80000DE044F400140AE044F4801401E044F40B
:105D900040147278824202D104F58014761C761C7D
:105DA000307866280BD013DC582877D009DC00281F
:105DB00075D04528F6D04628F4D047281AD19DE161
:105DC00018E0632835D0642879D0652812D195E190
:105DD000702873D008DC6728F1D069286FD06E284E
:105DE0000DD06F2806D1B5E073282CD0752875D05A
:105DF000782874D05A46179990476D1C75E1C4F302
:105E00000250022809D003280DD0D9F80010042828
:105E10000DD00D6009F1040967E1D9F80010EA1707
:105E2000C1E90052F6E7D9F800100D80F2E70D70D5
:105E3000F0E719F8041B8DF8001000208DF8010020
:105E4000EA46012003E059F804AB4FF0FF30610748
:105E50004FF0000102D40DE008F101018846B9427B
:105E60000FDA8045F8DB1AF808100029F4D108E0B1
:105E700008F1010188468142FADB1AF8081000296E
:105E8000F6D105985B46A0EB080721463846179ADD
:105E900000F094FA284400EB080507E04DE029E102
:105EA0000DE01AF8010B5A4617999047B8F101080E
:105EB000F7D25B4621463846179A13E142E00A22A0
:105EC0000092C4F302524FF0000A022A08D059F897
:105ED00004CB032A4FEAEC710AD00DE029E02AE056
:105EE00009F1070121F00702F2E802C1914609E039
:105EF0000FFA8CFC4FEAEC71042A03D14FFA8CFCA8
:105F00004FEAEC71002907DA0A460021DCF1000CA7
:105F100061EB02012D2202E0220504D52B228DF82F
:105F20000420012203E0E20701D02022F7E7904697
:105F300059E00A2102E010220DE010214FF0000A82
:105F400000910BE010224FF0000A44F004040827EF
:105F5000009203E008224FF0000A0092C4F30252BC
:105F6000022A05D059F804CB0021032A08D009E001
:105F700009F1070121F00702F2E802C1914605E0AC
:105F80001FFA8CFC042A01D10CF0FF0C4FF0000822
:105F9000220728D5702806D0009B83F0100353EA0F
:105FA0000A0305D00EE040228DF80420012208E00B
:105FB0005CEA010206D030228DF804208DF805003D
:105FC00002229046009B83F0080353EA0A030AD199
:105FD0005CEA010201D1620705D530228DF8042068
:105FE0004FF001087F1E582804D034A003900EA85B
:105FF00002900DE036A0F9E753466046009AFFF79D
:10600000DCFA84460398825C0298401E029002707B
:106010005CEA0100F0D1029806A9081A00F1200AF2
:10602000600702D524F4803400E00127574502DDE3
:10603000A7EB0A0000E0002000EB0A0100900598A1
:106040004144401A0590E00306D45B462146179A66
:10605000059800F0B3F90544002706E001A85A4668
:10606000C05D179990476D1C7F1C4745F6DBE00328
:106070000CD55B462146179A059800F09FF9054418
:1060800004E030205A46179990476D1C0099481E2D
:1060900000900029F5DC08E0029802995A46007841
:1060A000491C0291179990476D1CBAF10001AAF1A1
:1060B000010AF1DC65E100000928010030313233CA
:1060C0003435363738396162636465660000000034
:1060D000303132333435363738394142434445461E
:1060E0000000000000F058F90544761C30780028C4
:1060F0007FF4ECAD19B02846BDE8F08F620700D4FC
:10610000062709F1070222F0070CFCE80223E1460A
:1061100003F000485FEA080C02D00FF2702C0DE08B
:106120005FEA045C02D50FF2682C07E05FEAC47CEA
:1061300002D00FF2602C01E0AFF2700C4FF0FF388C
:1061400023F00043CDF850C065280CD006DC45286C
:1061500009D046281DD047283DD13DE0662818D0FB
:1061600067287ED138E00021112F01DB112000E0EB
:10617000781CCDE9000106A90EA8FFF7DDFCDDE9DA
:106180000F010E9A03910021009207F1010A049178
:106190004DE04FF000400097CDE9011006A90EA890
:1061A000FFF7CAFCDDE90F0203920E9B1199002252
:1061B000DDF80CA00093049211B9791C00EB010AE0
:1061C000B7EB0A0004D4C0F1FF3007F1010A0490D4
:1061D000AAEB0700019044E0012F00DA012700211B
:1061E000112F01DD112000E03846CDE9000106A99C
:1061F0000EA8FFF7A1FCDDE90F010E9A0391002123
:1062000004910092BA4621070CD40399514500DA53
:106210008A46BAF1010F05DD009AAAF10101515C2D
:10622000302908D0B84202DA10F1040F06DA012151
:10623000CDE9011015E0AAF10101E9E7002805DC2C
:10624000049901440491AAEB000102E0411C51456C
:1062500000DD8A460499401A401C01904FF000402E
:106260000290200704D40198504501DBCDF804804A
:1062700000208DF84F0002980DF14F07B0F1004F4C
:1062800025D02B200E9002984FF0020800280CDA3F
:10629000404202902D200E9007E00A210298FFF75D
:1062A00076F93031029007F8011DB8F10001A8F12C
:1062B0000108F2DC02980028EFD1791E0E980870D0
:1062C000307800F0200040F0450007F8020D12A8D9
:1062D000C01B00F107081498007800B1012000EB02
:1062E0000A01019801EBE07105984144401A401EF3
:1062F0000590E00306D45B462146179A059800F006
:106300005DF805441498007818B15A4617999047DB
:106310006D1CE00324D55B462146179A059800F0D2
:106320004DF805441CE00498002807DBDDE9030173
:10633000884203DD0098405C179901E017993020EE
:106340005A469047049805F10105401C04900198B5
:10635000401E019004D12E205A46179990476D1C7B
:10636000BAF10001AAF1010ADDDC05E017F8010B22
:106370005A46179990476D1CB8F10001A8F1010821
:10638000F4DC5B462146179A0598ABE62D00000029
:106390002B000000200000002DE9F04104460025FC
:1063A0001E461746880404D405E039462020B0472D
:1063B0006D1C641EF9D52846BDE8F0812DE9F04139
:1063C000044600251E469046C80301D5302700E04C
:1063D0002027880404D505E041463846B0476D1CA7
:1063E000641EF9D52846BDE8F0810A68531C0B608D
:1063F000107070470004000200018000400020007F
:10640000100008000400020000000080004000208E
:1064100000100008004000200010000800040002E6
:10642000406400080000002058000000185B0008CD
:106430009864000858000020B00E0000285B000897
:10644000030406080C1018203000000000010203AD
:106450000401020304060708090000000048E801DF
:10646000030406080C101820300000000000000093
:1064700000010203040607080900000000000000F4
:10648000000000000000000000000000000000000C
:086490000030000000000000D4
:0400000508000125C9
:00000001FF
